:200000001C222A3A1A023C00081422223E2222001E22221E22221E001C22020202221C00A0
:200020001E22222222221E003E02021E02023E003E02021E020202003C02020232223C0000
:200040002222223E222222001C08080808081C002020202020221C0022120A060A122200D6
:200060000202020202023E0022362A2A222222002222262A322222001C22222222221C0038
:200080001E22221E020202001C2222222A122C001E22221E0A1222001C22021C20221C0078
:2000A0003E080808080808002222222222221C0022222222221408002222222A2A36220012
:2000C000222214081422220022221408080808003E20100804023E003E06060606063E009C
:2000E00000020408102000003E30303030303E000000081422000000000000000000007F99
:2001000000000000000000000808080808000800141414000000000014143E143E14140093
:20012000083C0A1C281E08000626100804323000040A0A042A122C000808080000000000C1
:2001400008040202020408000810202020100800082A1C081C2A08000008083E08080000EF
:2001600000000000080804000000003E0000000000000000000008000020100804020000E7
:200180001C22322A26221C00080C080808081C001C22201804023E003E20101820221C0073
:2001A000101814123E1010003E021E2020221C003804021E22221C003E2010080404040079
:2001C0001C22221C22221C001C22223C20100E00000008000800000000000800080804003D
:2001E000100804020408100000003E003E00000004081020100804001C221008080008008B
:200200001C222A3A1A023C00081422223E2222001E22221E22221E001C22020202221C009E
:200220001E22222222221E003E02021E02023E003E02021E020202003C02020232223C00FE
:200240002222223E222222001C08080808081C002020202020221C0022120A060A122200D4
:200260000202020202023E0022362A2A222222002222262A322222001C22222222221C0036
:200280001E22221E020202001C2222222A122C001E22221E0A1222001C22021C20221C0076
:2002A0003E080808080808002222222222221C0022222222221408002222222A2A36220010
:2002C000222214081422220022221408080808003E20100804023E003E06060606063E009A
:2002E00000020408102000003E30303030303E000000081422000000000000000000007F97
:20030000040810000000000000001C203C223C0002021E2222221E0000003C0202023C00C7
:2003200020203C2222223C0000001C223E023C001824041E0404040000001C22223C201CA3
:2003400002021E222222220008000C0808081C00100018101010120C020222120E122200BB
:200360000C08080808081C000000362A2A2A220000001E222222220000001C2222221C0013
:2003800000001E22221E020200003C22223C202000003A060202020000003C021C201E00FF
:2003A00004041E04042418000000222222322C000000222222140800000022222A2A3600BF
:2003C000000022140814220000002222223C201C00003E1008043E00380C0C060C0C38008D
:2003E00008080808080808080E18183018180E002C1A000000000000002A142A142A000025
:00000001FF
